:100000000C9486050C94CE050C94CE050C94CE056C
:100010000C94CE050C94CE050C94CE050C94CE0514
:100020000C94CE050C94CE050C94AA0F0C94CE051E
:100030000C94BE1D0C94CE050C94CE050C94CE05EC
:100040000C94CE050C94CE050C94CE050C94CE05E4
:100050000C94CE050C94171E0C94CE050C94CE0572
:100060000C94CE050C9423080C94CE050C94CE056C
:100070000C94CE050C94CE050C94CE050C94CE05B4
:100080000C94CE050C94CE050C94CE050C94CE05A4
:100090000C94CE050C94CE050C94CE050C94CE0594
:1000A0000C94CE050C94CE050C94CE05F80D1F0EC5
:1000B000170F1F0E170F6B0E8E0E170FE50EF40E97
:1000C000F213F2132A142A14A514D914D016D01638
:1000D000F014D016811481148A16D0169F16BD16FE
:1000E0008800000000000000040005000600070072
:1000F000080009000A000B000C000D000E000F00A4
:100100001000110012001300140015001600170053
:10011000180019001A001B001C001D001E001F0003
:1001200020002100220023002400250026002700B3
:10013000280029002A002B002C002D002E002F0063
:10014000300031000000330034000000360037007A
:10015000380082003A003B003C003D003E003F007A
:1001600040004100420043004400450046000000BA
:10017000000049004A004E004C004D004B004F006B
:100180005000510052000000540055005600570026
:10019000580059005A005B005C005D005E005F0083
:1001A0006000610062006300000065008500670078
:1001B000680069006A000000000000000000000004
:1001C0000000000000000000890087008A008B000A
:1001D000E000E100E200E3000000E500E600E700E7
:1001E000291E1F20212223242526272D2E742A2B69
:1001F000141A0815171C180C12132F302804160790
:10020000090A0B0D0E0F3334311D1B061905111091
:10021000363738752C764E4B494C52504F514A4D1B
:1002200056545F6061555C5D5E57595A5B67626604
:100230006377444568696A807071727380806580F5
:1002400048463A3B3C3D3E3F4041424380808080AF
:100250007939007A7880807B7F7E8080807D808085
:10026000706339385F6C65643A20253032580A0073
:100270007573625F6C65643A20253032580A0073EA
:10028000656E6420253032583A20253032580A00F5
:1002900073656E642039443A20253032580A0025AF
:1002A000303258200073656E642037303A20253094
:1002B00032580A0073656E642039433A2025303283
:1002C000580A000A4B6579626F6172642073746129
:1002D00072742E0A000A55534220636F6E66696776
:1002E000757265642E0A000A0A544D4B3A3438641C
:1002F00036393634342B2F4C5546410A0A00300328
:10030000500043003900380020006B006500790080
:1003100062006F00610072006400200063006F00E3
:100320006E007600650072007400650072000000C7
:100330000E0374002E006D002E006B002E000000D6
:100340000403090409027400040100A03209040036
:1003500000010301010009211101000122400007F1
:1003600005810308000A09040100010301020009D4
:100370002111010001224D000705820308000A092E
:1003800004020001030000000921110100012236CE
:10039000000705830308000A0904030002030000A4
:1003A0000009211101000122220007058403200019
:1003B00001070504032000011201100100000008DC
:1003C000EDFE01980101010200010631FF0974A14F
:1003D000010975150026FF00952075088102097630
:1003E000150026FF00952075089102C005010980BF
:1003F000A10185021601002637001A81002AB700E4
:10040000751095018100C0050C0901A10185031635
:100410000100269C021A01002A9C02751095018198
:1004200000C005010902A1010901A1000509190186
:1004300029051500250195057501810295017503B2
:1004400081010501093009311581257F9502750863
:10045000810609381581257F950175088106050CEF
:100460000A38021581257F950175088106C0C005EF
:10047000010906A101050719E029E71500250195E5
:100480000875018102950175088101050819012986
:1004900005950575019102950175039101050719EF
:1004A0000029FF150026FF00950675088100C0632E
:1004B0006F6E73756D65723A20253034580A00737B
:1004C000797374656D3A20253034580A000A002586
:1004D00030325820006B6579626F6172643A200097
:1004E0004C45443A20253032580A0025583A2530E8
:1004F000386225730A000A20203031323334353611
:10050000370A00290A002575002F002575005D288F
:1005100000256400200025640020002564002000E0
:100520002564007C0025303258006D6F7573656B53
:100530006579205B62746E7C782079207620685D16
:10054000287265702F61636C293A205B006D6B5FC8
:10055000776865656C5F74696D655F746F5F6D6109
:1005600078203D2025640A006D6B5F776865656CB7
:100570005F6D61785F7370656564203D2025640A56
:10058000006D6B5F74696D655F746F5F6D6178207E
:100590003D2025640A006D6B5F6D61785F73706547
:1005A0006564203D2025640A006D6B5F696E74658B
:1005B0007276616C203D2025640A006D6B5F646576
:1005C0006C6179203D2025640A006D6B5F7768655A
:1005D000656C5F74696D655F746F5F6D6178203DF8
:1005E0002025640A006D6B5F776865656C5F6D61DF
:1005F000785F7370656564203D2025640A006D6B2B
:100600005F74696D655F746F5F6D6178203D202553
:10061000640A006D6B5F6D61785F7370656564205F
:100620003D2025640A006D6B5F696E7465727661AA
:100630006C203D2025640A006D6B5F64656C6179F8
:10064000203D2025640A000A00257500363A2077EF
:100650006865656C5F74696D655F746F5F6D617807
:100660003A20000A00257500353A20776865656CE8
:100670005F6D61785F73706565643A20000A0025DC
:100680007500343A2074696D655F746F5F6D6178D1
:100690003A20000A00257500333A206D61785F73B7
:1006A000706565643A20000A00257500323A2069B9
:1006B0006E74657276616C286D73293A20000A00A9
:1006C000257500313A2064656C6179282A31306DD6
:1006D00073293A20000A092D2056616C7565732034
:1006E0002D0A004D3E004D25643E20003F007365FD
:1006F000742064656661756C740A00433E2000775F
:10070000686572652064656C74613A206375727304
:100710006F723D25642C20776865656C3D25640A01
:1007200053656520687474703A2F2F656E2E776953
:100730006B6970656469612E6F72672F77696B6989
:100740002F4D6F7573655F6B6579730A000A092D0C
:10075000204D6F7573656B6579202D0A4553432FC6
:10076000713A09717569740A313A0964656C617985
:10077000282A31306D73290A323A09696E7465721C
:1007800076616C286D73290A333A096D61785F735D
:10079000706565640A343A0974696D655F746F5FEA
:1007A0006D61780A353A09776865656C5F6D6178C7
:1007B0005F73706565640A363A09776865656C5FD2
:1007C00074696D655F746F5F6D61780A0A703A09CC
:1007D0007072696E742076616C7565730A643A098B
:1007E0007365742064656661756C74730A75703A1C
:1007F000092B310A646F776E3A092D310A706775DB
:10080000703A092B31300A7067646F776E3A092DA0
:1008100031300A0A7370656564203D2064656C742C
:1008200061202A206D61785F7370656564202A20DD
:1008300028726570656174202F2074696D655F741E
:100840006F5F6D6178290A003F004D3E2000433EF6
:1008500020004C25640A000A092D20436F6E736F37
:100860006C65202D0A4553432F713A0971756974DF
:100870000A6D3A096D6F7573656B65790A000A092F
:100880002D204D61676963202D0A643A0964656211
:1008900075670A783A096465627567206D617472DC
:1008A00069780A6B3A096465627567206B657962DD
:1008B0006F6172640A6D3A096465627567206D6FD5
:1008C0007573650A763A0976657273696F6E0A7395
:1008D0003A097374617475730A633A09636F6E73CE
:1008E0006F6C65206D6F64650A302D343A096C6158
:1008F000796572302D34284631302D4634290A501E
:100900006175733A09626F6F746C6F616465720A26
:10091000003F0074696D65725F72656164333228EF
:10092000293A202530346C580A006B6579626F6172
:1009300072645F69646C653A2025580A006B6579BA
:10094000626F6172645F70726F746F636F6C3A2074
:1009500025580A00686F73745F6B6579626F617206
:10096000645F6C65647328293A2025580A000A09D7
:100970002D20537461747573202D0A004743433A48
:1009800020352E342E30204156522D4C4942433AC8
:1009900020322E302E30204156525F415243483A89
:1009A00020617672350A004F5054494F4E533A2019
:1009B0004C554641204D4F5553454B4559204558C0
:1009C0005452414B455920434F4E534F4C452043C1
:1009D0004F4D4D414E4420343039360A004255497E
:1009E0004C443A2034386436393634342B2028319C
:1009F000333A31343A32332044656320203920328F
:100A0000303230290A005649443A2030784645456C
:100A10004428742E6D2E6B2E29205049443A2030E4
:100A200078393830312850433938206B6579626F16
:100A300061726420636F6E766572746572292056E8
:100A400045523A203078303130310A004445534322
:100A50003A20636F6E766572747320504339382084
:100A60006B6579626F6172642070726F746F636F0F
:100A70006C20696E746F205553420A000A092D20BC
:100A800056657273696F6E202D0A000A6D6F75735B
:100A9000653A206F66660A000A6D6F7573653A20C5
:100AA0006F6E0A000A6B6579626F6172643A206F3B
:100AB00066660A000A6B6579626F6172643A206F3C
:100AC0006E0A000A6D61747269783A206F66660A70
:100AD000000A6D61747269783A206F6E0A000A64C8
:100AE000656275673A206F6E0A000A646562756711
:100AF0003A206F66660A000A0A626F6F746C6F6153
:100B00006465722E2E2E2000433E200011241FBE4D
:100B1000CFEFDAE0DEBFCDBF04B603FE28C0809180
:100B20005B0490915C04A0915D04B0915E048730F9
:100B3000904BA740B04BD9F410925B0410925C0428
:100B400010925D0410925E0414BE0FB6F894A8953E
:100B500080916000886180936000109260000FBEF9
:100B60001092010810920008E0E0F8E3099511E006
:100B7000A0E0B1E0E2E1FDE402C005900D92A833EF
:100B8000B107D9F724E0A8E3B1E001C01D92AB356D
:100B9000B207E1F70E940D0B0C9487260C9400001D
:100BA000FF93EF93E0913801F0913901309709F00C
:100BB0000995EF91FF910895FC018591803011F026
:100BC000EFDFFBCF0895FF27E0E230E247FF0CC0E4
:100BD000419597FF09C0EDE26095709580959095DD
:100BE000611D711D811D911D27FF02C0219530E3FC
:100BF00050E2AA27660F771F881F991FAA1FA41704
:100C000010F0A41B63955A95A9F7AA3008F0A95FC4
:100C1000A05DAF93F395611571058105910541F7CD
:100C2000ED3211F4EF93F395F21718F43F93F39527
:100C3000FBCF8F91B5DFFA95E1F70895E991F9912E
:100C40008591803021F0853219F0AADFF9CF08951F
:100C500020E0E89455915532C1F3503311F4689473
:100C600055915A3348F4505390F3220F022E220F1D
:100C7000220F200D250FF4CF0EF421958991999123
:100C8000533619F3533729F1533559F1BC018827ED
:100C90009927E8945C3621F489919991689455914B
:100CA000543639F446EF7EF077FF0DC08FEF9FEF9B
:100CB0000AC055374AE039F0583540E121F0523644
:100CC00042E009F00895FF93EF937DDFEF91FF91EC
:100CD000B7CFFF93EF93FC0181918030B9F360DFD0
:100CE000FBCFFF93EF9368DFF1CFDF93CF93CDB7C7
:100CF000DEB72596A3DFCF91DF9108955C9AEFE9E7
:100D0000FFE03197F1F700C000000E941C088FE956
:100D10009FE00197F1F700C000005C980895CF9321
:100D2000CFEF0E940808C1508F3FFFEF9F0741F4AB
:100D3000EFE9FFE03197F1F700C00000C111F1CFFA
:100D4000CF910895EF92FF920F931F93CF93DF936C
:100D5000539A549A519A5B9A5C9A599A0E94F20754
:100D60005C9A5B9820E52A95F1F75B9A8FEF90E704
:100D700022E0815090402040E1F700C0000004EBE9
:100D800012E085EAE82E82E0F82E8CE90E947E06C9
:100D90000E948F06EC01CF3F8FEFD80719F4EBE3E9
:100DA000F1E02DC080913D0480FF0AC0DF93CF9316
:100DB0001F930F930E9475060F900F900F900F9046
:100DC000CA3FD10561F780E70E947E060E948F0628
:100DD000EC01CF3F8FEFD807C1F280913D0480FF37
:100DE0000AC0DF93CF93FF92EF920E9475060F9097
:100DF0000F900F900F90CA3FD10539F6D0CF1192C6
:100E000081E0EB34F807D9F75C98DF91CF911F911F
:100E10000F91FF90EF900895EF92FF920F931F9321
:100E2000CF93DF930E940808F82E082F192F0F3F49
:100E30008FEF180709F04EC080913A01882309F41A
:100E400093C000E912E09FE7E92E92E0F92E8DE9C8
:100E50000E947E060E948F06EC01CF3F8FEFD807DD
:100E600021F410923A0180E07FC080913D0480FF20
:100E70000AC0DF93CF931F930F930E9475060F90C4
:100E80000F900F900F90CA3FD10559F780913A010A
:100E90000E947E060E948F06EC01CF3F8FEFD8079D
:100EA000B1F280913D0480FF10C0DF93CF93809119
:100EB0003A011F928F93FF92EF920E9475060F9056
:100EC0000F900F900F900F900F90CA3FD10509F02F
:100ED000BECFC7CF80913D0480FF0CC09F93FF928F
:100EE0008FE992E09F938F930E9475060F900F9069
:100EF0000F900F90E80183E0D695C7958A95E1F7AA
:100F00006F2D67708C2F8F7007FF14C00E94FF1128
:100F1000882319F1CF70DD27C55CDE4F07701127DC
:100F200081E090E001C0880F0A95EAF780959881EA
:100F3000892312C00E94FF1181110FC0CF70DD27DD
:100F4000C55CDE4F0770112781E090E001C0880F7B
:100F50000A95EAF79881892B88835C9A8AE68A95B4
:100F6000F1F700C05C988F2DDF91CF911F910F9109
:100F7000FF90EF900895E82FF0E0E55CFE4F808150
:100F8000089580FD02C090E701C091E790933A0177
:100F900081FF05C090913A01946090933A0190913D
:100FA0003D0490FF0CC01F928F9380E792E09F93C7
:100FB0008F930E9475060F900F900F900F90809165
:100FC0003D0480FF0EC080913A011F928F9380E60E
:100FD00092E09F938F930E9475060F900F900F9051
:100FE0000F90089583E38093CC001092CD00E9EC3C
:100FF000F0E0808180698083808188608083EAEC72
:10100000F0E080818063808352985A9A78940895A2
:1010100020914B0180914C01821759F030E0F90189
:10102000E35BFE4F80812F5F3F4F20934B0190E0A9
:1010300008958FEF9FEF08959091C80095FFFCCF22
:101040008093CE0008951F920F920FB60F92112435
:101050002F933F934F938F939F93EF93FF938091A1
:101060004C0190E09C012F5F3F4F40914B01421794
:1010700041F03091CE00FC01E35BFE4F30832093C2
:101080004C01FF91EF919F918F914F913F912F9143
:101090000F900FBE0F901F901895809159030895DF
:1010A000CF93DF9300D01F92CDB7DEB79C01809124
:1010B0005204843019F593E099833B832A839093FB
:1010C000E9008FEF9091E800815095FD06C095ED05
:1010D0009A95F1F700008111F5CF8091E80085FF26
:1010E0000DC040E050E063E070E0CE0101960E9448
:1010F000C30C8091E8008E778093E8000F900F90EA
:101100000F90DF91CF910895CF93DF9300D01F927E
:10111000CDB7DEB720915204243031F522E0298387
:10112000805891099B838A8383E08093E9008FEF45
:101130009091E800815095FD06C095ED9A95F1F7E4
:1011400000008111F5CF8091E80085FF0DC040E0DF
:1011500050E063E070E0CE0101960E94C30C8091E4
:10116000E8008E778093E8000F900F900F90DF914A
:10117000CF910895209152042430F1F422E020937D
:10118000E9002FEF3091E800215035FD06C035ED24
:101190003A95F1F700002111F5CF2091E80025FFE5
:1011A0000BC040E050E065E070E00E94C30C80910D
:1011B000E8008E778093E8000895CF93DF93209125
:1011C0005204243049F521E02093E90021E8215020
:1011D00059F03091E80035FD07C0EFE3F1E03197B9
:1011E000F1F700C00000F3CF2091E80025FF14C004
:1011F000EC0140E050E068E070E00E94C30C809198
:10120000E8008E778093E80088E0FE01A1E5B3E076
:1012100001900D928A95E1F7DF91CF910895CF93D8
:10122000C0914F02C1110BC00E94FC1D643C79406B
:101230008105910520F081E080934F02C1E08C2F61
:10124000CF910895FF920F931F93CF93DF93D82FE1
:101250000FB607FE83C080915204843081F08091E4
:10126000030190E001962091050130E08223932351
:101270002091040130E08217930709F0CDC00E944D
:101280000F09811110C08091030190E00196209117
:10129000050130E0822393232091040130E082177E
:1012A000930709F0B9C00E94F01D8C01C091E900BC
:1012B000CF709091EC00892F817090FD80E8C82B51
:1012C00084E08093E90085E0F82E8091EB0085FDB5
:1012D00042C08091EB0080FF3EC08091EE0087FF0E
:1012E0003AC08091040190910301981709F457C006
:1012F0009091E80095FF8EC0E0910101F09102010C
:10130000E80FF11D20818F5F909105018923809363
:1013100004012093F1008091E80085FDE2CF8091E7
:10132000E80080FFDECF8091E8008E778093E800B0
:10133000F0920001D6CF8091030190E001962091B8
:10134000050130E0822393232091040130E08217CD
:10135000930709F44CC0CF70C093E900409103019A
:10136000842F90E001962091050130E082239323A1
:101370002091040130E08217930709F450C0E091F6
:101380000101F0910201E40FF11DD083809103016E
:101390008F5F9091050189238093030140C0809164
:1013A000E80085FF37C0D093F10021E03091F300D1
:1013B0008091F20090E0932B892B91F08091E800CE
:1013C00080FF0EC08091E80085FF03C01092F100FD
:1013D000F9CF8091E8008E778093E800F0920001C9
:1013E000222309F4A8CFCF70C093E90018C08091E0
:1013F0000001882309F4AFCF0E94F01D9C018017E3
:10140000910711F4890161CF90910001915090935F
:101410000001F8CF20E0CACF40910301B0CF80E0B7
:10142000DF91CF911F910F91FF900895809151040A
:10143000811104C00E942F0F0C948C0F08951092FC
:1014400051040895089542E061EC81E00E943C0C53
:1014500042E061EC82E00E943C0C42E061EC83E0FF
:101460000E943C0C42E261EC84E00C943C0C8091C4
:101470005404833009F453C030F4813071F0823069
:1014800009F48CC008958A3009F478C08B3009F4CF
:101490005EC0893009F09AC020C080915304813A1F
:1014A00009F094C08091E800877F8093E8008091E4
:1014B000570490915804892B21F468E081E593E06A
:1014C00003C060E080E090E070E00E94100D809129
:1014D000E8008B778093E80008958091530481326F
:1014E00009F074C08091570490915804892B09F039
:1014F0006DC08091E800877F8093E8008091E800CC
:1015000082FD05C0809152048111F8CF5FC08091A7
:10151000F100809359038091E8008B7753C080914C
:101520005304813A09F052C08091570490915804B5
:10153000892B09F04BC08091E800877F8093E800F9
:101540008091E80080FFFCCF8091100136C080912F
:1015500053048132D9F58091570490915804892B16
:10156000A9F58091E800877F8093E8000E94710CC4
:1015700080915504809310010C94A2138091530420
:10158000813221F58091E800877F8093E8000E94F6
:10159000710C8091560480935A03089580915304EE
:1015A000813AA1F48091E800877F8093E8008091E0
:1015B000E80080FFFCCF80915A038093F100809176
:1015C000E8008E778093E8000C94710C0895809168
:1015D000590380935002109259030E94FD110C94FC
:1015E000A2130C94E70A0E947D1D80915004882369
:1015F00029F00E94A61D81110C94260C08950E94CA
:10160000BA1D809150028093590308950C94FF0AEB
:1016100008950C94080B0C94080BCF9384B7877F24
:1016200084BF0FB6F894A89580916000886180937C
:101630006000109260000FBE90E080E80FB6F89452
:1016400080936100909361000FBE82E299E00E9456
:10165000501D86E091E00E94931087EE92E00E9478
:10166000DC050E940B0B0E9452110E942F0F0E945A
:101670008C0F78940E94541180915204843029F088
:101680000E9478100E94080BF7CF85ED92E00E942F
:10169000DC050E94090B83EC92E00E94DC05C4E0AB
:1016A00080915204853019F40E94F30AF9CF0E9408
:1016B00058112091E4003091E50080914D02909105
:1016C0004E022817390709F468C08091E400909110
:1016D000E50090934E0280934D020E940F098823EB
:1016E00009F45BC080915204843009F056C08091A7
:1016F000E9008F702091EC00922F917020FD90E80E
:10170000892BC093E9009091EB0090FF43C090912A
:10171000EE0097FF3FC0909104012091030129172B
:1017200009F12091E80025FF1DC0E0910101F09131
:101730000201E90FF11D30819F5F20910501922385
:10174000909304013093F1009091E80095FDE3CF70
:101750009091E80090FFDFCF9091E8009E77909302
:10176000E800D9CF9091F3002091F20030E0392BBE
:10177000232B81F09091E80090FF0CC09091E8003D
:1017800095FF03C01092F100F9CF9091E8009E7789
:101790009093E8008F708093E9000E94781080CFCA
:1017A000292F332723303105C9F060F4213031056A
:1017B00081F02230310509F041C084E790E024E453
:1017C00033E040C021323105E1F02232310531F100
:1017D00035C082E190E028EB33E034C099278130B6
:1017E000910549F028F0029749F5EEEFF2E005C0C7
:1017F000E0E4F3E002C0E0E3F3E0849190E09F01D5
:1018000021C064307105D0F4660F771FFB01EB5DDA
:10181000FE4F2081318189E090E014C06430710571
:1018200068F4FB01EE0FFF1FE35EFE4F2081318164
:10183000FB01E75EFE4F808190E004C080E090E015
:1018400020E030E0FA0131832083089580E189BDF2
:1018500082E189BD09B400FEFDCF8091D8008F7D63
:101860008093D8008091E00082608093E0008091B6
:10187000E00081FDFCCF0895982F973068F5909394
:10188000E900981739F07091EC002091ED0050912B
:10189000F00003C0242F762F50E021FD02C09F5F8F
:1018A000ECCF3091EB003E7F3093EB003091ED00B8
:1018B0003D7F3093ED003091EB0031603093EB00D1
:1018C0007093EC002093ED005093F0002091EE0017
:1018D00027FDE5CF80E008958F708093E90081E0D7
:1018E00008958091530487FF11C08091E80082FD24
:1018F00005C0809152048111F8CF11C08091E80099
:101900008B770BC080915204882349F08091E800C6
:1019100080FFF8CF8091E8008E778093E8000895EB
:101920002091E4003091E50095E64091EC00842F91
:10193000817040FF23C08091E80080FD1DC0809130
:101940005204882399F0853099F08091EB0085FD51
:1019500011C04091E4005091E5002417350729F3A8
:10196000915011F09A01E1CF84E0089582E008954A
:1019700083E0089581E0089580E008954091E800B3
:1019800042FFDDCF0895CF92DF92EF92FF920F9347
:101990001F93CF93DF93EC018B017A010E94900C8F
:1019A000811135C0E114F10439F0F7018081918192
:1019B000081B190BC80FD91FC12CD12C01151105FB
:1019C00029F18091E80085FD18C08091E8008E77AC
:1019D0008093E8000E947810E114F10449F0F701C7
:1019E00080819181C80ED91ED182C08285E00FC04E
:1019F0000E94900C882311F30AC089918093F10012
:101A000001501109FFEFCF1ADF0AD8CF80E0DF9134
:101A1000CF911F910F91FF90EF90DF90CF9008959D
:101A20002091590430915A042617370748F0611560
:101A3000710539F42091E8002E772093E80001C069
:101A4000B901FC0120E06115710579F18091520422
:101A50008823F1F18530F1F18091E80083FD3CC0ED
:101A60008091E80082FD2EC08091E80080FFEBCFDE
:101A70002091F3008091F20090E0922B61157105A6
:101A800051F08830910538F421912093F100615094
:101A900071090196F3CF21E0089709F020E08091C9
:101AA000E8008E778093E800CECF2111CFCF0AC017
:101AB00080915204882361F0853061F08091E800C4
:101AC00083FD0AC08091E80082FFF2CF80E0089594
:101AD00082E0089583E0089581E0089520915904FB
:101AE00030915A042617370748F06115710539F40B
:101AF0002091E8002E772093E80001C0B901FC0195
:101B000020E06115710591F180915204882309F458
:101B100040C0853009F43FC08091E80083FD3DC09E
:101B20008091E80082FD2FC08091E80080FFE9CF1E
:101B30002091F3008091F20090E0922B61157105E5
:101B400059F08830910540F424912093F1003196AA
:101B5000615071090196F2CF21E0089709F020E069
:101B60008091E8008E778093E800CBCF2111CCCF15
:101B70000AC080915204882361F0853061F0809121
:101B8000E80083FD0AC08091E80082FFF2CF80E088
:101B9000089582E0089583E0089581E008951F93F9
:101BA000CF93DF93CDB7DEB7AA970FB6F894DEBF19
:101BB0000FBECDBFE3E5F4E08091F100819324E016
:101BC000EB35F207C9F70E94370A8091E80083FFDE
:101BD0002EC18091530490915404492F50E04A3013
:101BE000510508F024C1FA01EA5AFF4F0C946D2602
:101BF000803821F0823809F01AC108C080914F0462
:101C000090915004992389F082600FC0809157040D
:101C10008F70873008F00BC18093E9008091EB0052
:101C200085FB882780F91092E9009091E800977F62
:101C30009093E8008093F1001092F100D1C0282F1A
:101C40002D7F09F0F4C0882319F0823061F0EFC0D5
:101C500080915504813009F0EAC0933009F080E0AA
:101C6000809350042EC08091550481112AC0809128
:101C700057048F702FEF280F263008F0D8C08093BC
:101C8000E9002091EB0020FF1CC0933021F48091EB
:101C9000EB00806214C09091EB0090619093EB0098
:101CA00021E030E0A90102C0440F551F8A95E2F7F8
:101CB0004093EA001092EA008091EB0088608093E4
:101CC000EB001092E9008091E800877F8093E800A4
:101CD0000E94710CACC08111AAC0109155041F77ED
:101CE0008091E3008078812B8093E3008091E8006D
:101CF000877F8093E8000E94710C8091E80080FF4C
:101D0000FCCF8091E30080688093E300111102C052
:101D100082E001C083E08093520489C08058823001
:101D200008F085C080915504909156048C3D53E095
:101D3000950779F583E08A838AE289834FB7F8941F
:101D4000DE01139620E03EE051E2E32FF0E05093F5
:101D50005700E49120FF03C0E295EF703F5FEF7002
:101D60008E2F90E0EA3010F0C79601C0C0968D9398
:101D70009D932F5F243149F74FBF8091E800877F03
:101D80008093E8006AE270E0CE0101960E94100D97
:101D900016C06091570470915804AE014F5F5F4FB9
:101DA0000E94D00BBC01892B09F441C09091E8003E
:101DB000977F9093E80089819A810E946E0D8091AF
:101DC000E8008B778093E80032C0803881F58091FD
:101DD000E800877F8093E80080914E048093F100B3
:101DE0008091E8008E7772CF811121C080915504D7
:101DF0009091560499270297D4F48091E800877F48
:101E00008093E8008091550480934E040E94710CE9
:101E100080914E04811106C08091E30087FD02C0CD
:101E200081E001C084E0809352040E94230A8091E3
:101E3000E80083FF0AC08091E800877F8093E80074
:101E40008091EB0080628093EB00AA960FB6F89425
:101E5000DEBF0FBECDBFDF91CF911F9108950E94CD
:101E60009D0F0E94A50FE0EEF0E0808181608083ED
:101E7000E8EDF0E080818F77808319BCA7EDB0E0BA
:101E80008C918E7F8C9380818F7E80831092510401
:101E900008950F931F93CF93DF930E949D0F0E948D
:101EA000A50FC8EDD0E088818F778883888180680E
:101EB000888388818F7D888319BC10925204109288
:101EC0004E041092500410924F0400EE10E0F801FE
:101ED00080818B7F808388818160888342E060E09D
:101EE00080E00E943C0CE1EEF0E080818E7F8083F8
:101EF000E2EEF0E080818160808380818860808371
:101F0000F80180818E7F8083888180618883DF9162
:101F1000CF911F910F910895E8EDF0E080818F7EC1
:101F20008083E7EDF0E080818160808384E082BF80
:101F300081E0809351040C94490FE8EDF0E080813A
:101F40008E7F80831092E20008951092DA00109242
:101F5000E10008951F920F920FB60F9211242F9354
:101F60003F934F935F936F937F938F939F93AF9321
:101F7000BF93EF93FF938091E10082FF0BC08091AC
:101F8000E20082FF07C08091E1008B7F8093E10037
:101F90000E9477108091DA0080FF1FC08091D800E6
:101FA00080FF1BC08091DA008E7F8093DA008091E1
:101FB000D90080FF0DC080E189BD82E189BD09B4EF
:101FC00000FEFDCF81E0809352040E94160A05C0F6
:101FD00019BC109252040E941F0A8091E10080FFF8
:101FE00019C08091E20080FF15C08091E2008E7FD1
:101FF0008093E2008091E20080618093E200809112
:10200000D80080628093D80019BC85E08093520488
:102010000E94F10A8091E10084FF30C08091E200CB
:1020200084FF2CC080E189BD82E189BD09B400FE36
:10203000FDCF8091D8008F7D8093D8008091E10002
:102040008F7E8093E1008091E2008F7E8093E2009A
:102050008091E20081608093E20080914E048823A9
:1020600011F084E007C08091E30087FD02C081E0A9
:1020700001C083E0809352040E94060B8091E1002E
:1020800083FF24C08091E20083FF20C08091E100A3
:10209000877F8093E10082E08093520410924E0487
:1020A0008091E1008E7F8093E1008091E2008E7F3D
:1020B0008093E2008091E20080618093E20042E040
:1020C00060E080E00E943C0C0E94220AFF91EF91A8
:1020D000BF91AF919F918F917F916F915F914F9140
:1020E0003F912F910F900FBE0F901F90189508955C
:1020F000CF93809152048823A1F0C091E900CF7062
:102100009091EC00892F817090FD80E8C82B10928F
:10211000E9008091E80083FD0E94CF0DCF70C0934D
:10212000E900CF9108959093600380935F03089531
:10213000E0915F03F0916003309721F00190F0810E
:10214000E02D099480E00895EF92FF920F931F9382
:10215000CF93DF93E0915F03F09160033097B1F18B
:102160008C010280F381E02D099580913D0482FF6E
:102170002DC080FF04C085ED94E00E94DC05E801DD
:1021800018E08FECE82E84E0F82E80913D0480FF6B
:102190000BC088811F928F93FF92EF920E94750669
:1021A0000F900F900F900F90115021961111EDCFBD
:1021B00080913D0480FF0AC08DEC94E0DF91CF91C7
:1021C0001F910F91FF90EF900C94DC05DF91CF9160
:1021D0001F910F91FF90EF900895E0915F03F091B0
:1021E0006003309721F00480F581E02D0994089573
:1021F000CF93DF9320915D0330915E032817390759
:1022000009F190935E0380935D03E0915F03F09189
:1022100060033097B9F0EC010680F781E02D099555
:1022200080913D0482FF0EC080FF0CC0DF93CF93EE
:102230008FEB94E09F938F930E9475060F900F9001
:102240000F900F90DF91CF910895CF93DF9320915E
:102250005B0330915C032817390709F190935C0305
:1022600080935B03E0915F03F09160033097B9F0D6
:10227000EC010084F185E02D099580913D0482FFF9
:102280000EC080FF0CC0DF93CF938FEA94E09F9342
:102290008F930E9475060F900F900F900F90DF9113
:1022A000CF9108950C94FE110E94E71D0C94A20694
:1022B000BF92CF92DF92EF92FF920F931F93CF9333
:1022C000DF9300D000D01F92CDB7DEB70E940C077D
:1022D00002E613E0F12C8F2D0E94BB07B82EF80107
:1022E000C080C82639F4F3940F5F1F4FF0E1FF124E
:1022F000F2CF30C080913D0481FD0E941312D12C99
:10230000EE24E3948C2D8E21F9F0D982FA8291E0AB
:102310008B2D8E2109F490E09B830E94F01D81603B
:10232000782F9D838C8349815A816B818D810E9496
:10233000491249815A816B817C818D810E94681D7F
:10234000F80180818E258083D394EE0CF8E0DF12B3
:10235000D9CFC9CF8FEF89838A831B820E94F01D5A
:102360008160782F9D838C8349815A816B818D8117
:102370000E9449120E94671D0E9494200E9498109A
:1023800090916103891741F10E9498108093610335
:1023900090913D0492FF0EC090FF0CC01F928F934E
:1023A00080EE94E09F938F930E9475060F900F909C
:1023B0000F900F90809161030F900F900F900F90EE
:1023C0000F90DF91CF911F910F91FF90EF90DF90D1
:1023D000CF90BF900C94791D0F900F900F900F909D
:1023E0000F90DF91CF911F910F91FF90EF90DF90B1
:1023F000CF90BF9008950C94C10708950895CF938E
:10240000C62F0E94BB0721E030E002C0220F331F1D
:10241000CA95E2F790E02823392381E0232B09F4C1
:1024200080E0CF910895EF92FF920F931F93CF9387
:10243000DF9386EF94E00E94DC05C0E0D0E08DE2FF
:10244000E82E81E0F82E0BEE14E08C2F0E94BB07E3
:102450000E94551DFF92EF921F928F93DF93CF93AF
:102460001F930F930E94750621968DB79EB708960D
:102470000FB6F8949EBF0FBE8DBFC031D10529F7AE
:10248000DF91CF911F910F91FF90EF9008950895E4
:102490000895CF93DF93CDB7DEB72B970FB6F8949F
:1024A000DEBF0FBECDBF942F4F83252F588769877E
:1024B0007A878B874A855B85452B31F02F3F31F436
:1024C00081E09F3F19F403C081E001C080E080FDFE
:1024D00007C04F81588569857A858B850E94681D64
:1024E000DE01119686E0FD0111928A95E9F785E0FB
:1024F000FE01379601900D928A95E1F749815A8144
:102500006B817C818D819E810E94CA192B960FB6AA
:10251000F894DEBF0FBECDBFDF91CF910895CF936A
:10252000DF93882309F48FC0C82F8EE78C0F833088
:1025300018F5C23829F0C33831F0C4E0D7E405C03B
:10254000C2E0D9E302C0C1E0D3E50E9498108C2319
:1025500009F079C08D2F0E94B21C0E942A1D2FEF16
:1025600081EE94E0215080409040E1F700C00000EF
:102570008D2F0E94CF1C10C08CEF8C0F813A20F061
:1025800080E58C0F8E3260F48C2F0E94BE23811167
:102590005AC08C2F0E94B21CDF91CF910C942A1D3F
:1025A00080E28C0F883048F4C77081E001C0880F4A
:1025B000CA95EAF70E94F01CEFCF8BE58C0F8330B1
:1025C00080F4C53A29F0C63A31F083E890E005C0BE
:1025D00081E890E002C082E890E0DF91CF910C9416
:1025E000F81088E58C0F873170F5C83A89F0C93A40
:1025F00091F0CA3A99F0CB3AA1F0CC3AA9F0CD3A91
:10260000B1F0CE3AB9F0CF3AC1F080E090E017C017
:1026100082EE90E014C089EE90E011C08AEE90E066
:102620000EC085EB90E00BC086EB90E008C083EB1A
:1026300090E005C084EB90E002C087EB90E0DF9172
:10264000CF910C942511DF91CF910895CF93DF9313
:10265000882309F454C09EE7980F933008F5823818
:1026600029F0833831F0C4E0D7E405C0C2E0D9E3F3
:1026700002C0C1E0D3E50E9498108C2309F43FC04A
:102680008D2F0E94B21C0E942A1D2FEF81EE94E034
:10269000215080409040E1F700C000008D2F08C01D
:1026A0009CEF980F913A20F090E5980F9E3218F425
:1026B0000E94CF1C0DC090E2980F983068F487708C
:1026C00091E001C0990F8A95EAF7892F0E94F61CC4
:1026D000DF91CF910C942A1D9BE5980F933030F435
:1026E00080E090E0DF91CF910C94F810885A873108
:1026F00030F480E090E0DF91CF910C942511DF91D0
:10270000CF910895882321F00E94F01C0C942A1D7B
:102710000895882321F00E94F61C0C942A1D089528
:102720000E94101D0E94DF1C0E942A1D0E94392158
:102730000E94072080E090E00E94F81080E090E086
:102740000C9425110E94001D0C949013CF92DF92DF
:10275000EF92FF920F931F93CF93DF9300D000D09F
:102760001F92CDB7DEB76C010E947B1D811118C38B
:1027700085E0F601DE01119601900D928A95E1F750
:10278000F60140815181238134812115310531F0D9
:102790005F3F31F481E04F3F19F403C081E001C095
:1027A00080E080FDFDC2F601F280E580E2948FE0DA
:1027B000E82249835A83FB82722F3D832C836F2D3D
:1027C0008D810E942E1C8C010E942D1C0E941D1BBD
:1027D000E12FE295EF708E2F90E0FC01E05AFF4F61
:1027E0000C946D26812F807F1F70882311F0129525
:1027F000107FFF20B9F0112329F0812F0E94031DC3
:102800000E942A1D802F0F900F900F900F900F9015
:10281000DF91CF911F910F91FF90EF90DF90CF90BC
:102820000C948F12802F0E942613112309F4B8C232
:10283000812F0E94091D0F900F900F900F900F9005
:10284000DF91CF911F910F91FF90EF90DF90CF908C
:102850000C942A1D812F807F1F70803211F01295F9
:10286000107F002319F0013009F12BC0FF20A9F0DF
:10287000EE2059F1F1E0812FEF1228C00F900F9058
:102880000F900F900F90DF91CF911F910F91FF90BC
:10289000EF90DF90CF900C94131DEE2021F021E0FB
:1028A000E21609F47DC20E94161D4DC0FF20E9F01A
:1028B00085E08E1508F474C20E94ED1C812329F076
:1028C00042C0FF20F1F1E11015C0812F0F900F9051
:1028D0000F900F900F90DF91CF911F910F91FF906C
:1028E000EF90DF90CF900C94821394E09E1508F443
:1028F00057C229C0F601858180FF13C08F70858380
:10290000E4CF003F09F489C108F055C180E4800F8D
:10291000803208F459C1FF2009F4EAC1EE2009F41D
:102920009AC1802F0E948F12093309F0DAC1FFEF9C
:1029300021EE84E0F15020408040E1F700C000002B
:102940002FC2E110D7C1812F59C1812F869586955D
:10295000837019F08130B9F023C2FF2019F0C8014B
:10296000937002C080E090E00F900F900F900F9056
:102970000F90DF91CF911F910F91FF90EF90DF901B
:10298000CF900C94F810FF2019F0C801937002C08A
:1029900080E090E00F900F900F900F900F90DF91DC
:1029A000CF911F910F91FF90EF90DF90CF900C94FB
:1029B0002511802FFF2019F00E941A1F02C00E94CB
:1029C000821F0F900F900F900F900F90DF91CF917B
:1029D0001F910F91FF90EF90DF90CF900C94072004
:1029E000812F837009F070C0F110DAC1202F229579
:1029F00026952770220F220F602F6F70862F90E090
:102A0000A0E0B0E06C017D01022E04C0CC0CDD1C06
:102A1000EE1CFF1C0A94D2F704FF12C08FE090E076
:102A2000A0E0B0E004C0880F991FAA1FBB1F2A9521
:102A3000D2F7BC01CD01609570958095909503C04B
:102A400060E070E0CB011695169513701230B1F06E
:102A500040F56C297D298E299F29113031F10F9085
:102A60000F900F900F900F90DF91CF911F910F91CA
:102A7000FF90EF90DF90CF900C94421B6C297D2942
:102A80008E299F290F900F900F900F900F90DF913C
:102A9000CF911F910F91FF90EF90DF90CF900C940A
:102AA0005C1B0E94421BC701B6010F900F900F9054
:102AB0000F900F90DF91CF911F910F91FF90EF90AA
:102AC000DF90CF900C94281BFF2019F0812F81708C
:102AD00001C08695882309F463C1202F229526958D
:102AE0002770220F220F602F6F70862F90E0A0E0DA
:102AF000B0E06C017D01022E04C0CC0CDD1CEE1C8C
:102B0000FF1C0A94D2F704FF12C08FE090E0A0E00F
:102B1000B0E004C0880F991FAA1FBB1F2A95D2F7E7
:102B2000BC01CD01609570958095909503C060E0E3
:102B300070E0CB011695169513701230B1F040F588
:102B40006C297D298E299F29113031F10F900F902A
:102B50000F900F900F90DF91CF911F910F91FF90E9
:102B6000EF90DF90CF900C94091C6C297D298E2961
:102B70009F290F900F900F900F900F90DF91CF91A2
:102B80001F910F91FF90EF90DF90CF900C941B1C42
:102B90000E94091CC701B6010F900F900F900F9073
:102BA0000F90DF91CF911F910F91FF90EF90DF90E9
:102BB000CF900C94F71B023F09F45EC008F449C0A3
:102BC000033F09F46CC0A7CE902F9071E92E812F9E
:102BD0008F71FF2051F00E94901B802FEE2019F082
:102BE0008295807F73CE8F7071CE0E94B11B802F33
:102BF000EE2019F08295807F01C08F700F900F90AA
:102C00000F900F900F90DF91CF911F910F91FF9038
:102C1000EF90DF90CF900C948913FF20A9F0E4E0AF
:102C2000EE1508F4BDC0812F8F710F900F900F909B
:102C30000F900F90DF91CF911F910F91FF90EF9028
:102C4000DF90CF900C94D61BF5E0FE1508F4A8C0D9
:102C5000EACFFF2099F0812F8F710F900F900F9086
:102C60000F900F90DF91CF911F910F91FF90EF90F8
:102C7000DF90CF900C94901BFF2069F3812F8F7110
:102C80000F900F900F900F900F90DF91CF911F91A9
:102C90000F91FF90EF90DF90CF900C94B11BFF202D
:102CA00089F0812F8F710F900F900F900F900F90E0
:102CB000DF91CF911F910F91FF90EF90DF90CF9018
:102CC0000C947B1B0F900F900F900F900F90DF9143
:102CD000CF911F910F91FF90EF90DF90CF900C94C8
:102CE000761B033509F423CE073409F059C01FCEF3
:102CF000EE2021F2802F0F900F900F900F900F90E9
:102D0000DF91CF911F910F91FF90EF90DF90CF90C7
:102D10000C942613412F4F70602FC6010E94941E01
:102D20000F900F900F900F900F90DF91CF911F9108
:102D30000F91FF90EF90DF90CF900C94781A0111D3
:102D40002FC0FF2069F10E94A2132FEF80E792E0CD
:102D5000215080409040E1F700C000000F900F909C
:102D60000F900F900F90DF91CF911F910F91FF90D7
:102D7000EF90DF90CF900C943D1E412F4F70602F4D
:102D8000C6010F900F900F900F900F90DF91CF9191
:102D90001F910F91FF90EF90DF90CF900C94971EB2
:102DA0000F900F900F900F900F90DF91CF911F9188
:102DB0000F91FF90EF90DF90CF9008951F93CF93E6
:102DC000DF9300D000D01F92CDB7DEB7942F498398
:102DD000252F5A836B837C838D834C815D81452BAA
:102DE00031F02F3F31F481E09F3F19F403C081E0BF
:102DF00001C080E0182F117080FD31C049815A81D7
:102E00006B817C818D810E942E1C292F22952F7031
:102E10002C3030F42A30A0F42250223030F022C07E
:102E20002C30C9F02F30B9F01DC0853A28F4843019
:102E3000C0F4823028F415C090E2980F983088F0E2
:102E4000883E30F4803E68F48450813A58F409C0DA
:102E5000803F41F406C093FB112710F903C010E036
:102E600001C011E0812F0F900F900F900F900F90E5
:102E7000DF91CF911F910895CF93DF9300D000D0C1
:102E80001F92CDB7DEB70F900F900F900F900F905D
:102E9000DF91CF910895CF93DF9300D000D000D081
:102EA000CDB7DEB726960FB6F894DEBF0FBECDBF06
:102EB000DF91CF9108951F93CF93DF93C091720359
:102EC00016E080917303C81799F0D0E01C9FF001C1
:102ED0001D9FF00D1124EC58FC4F408151816281FF
:102EE0007381848195810E944B172196C770E9CF29
:102EF000DF91CF911F9108954091A4035091A503B4
:102F00006091A6037091A7038091A8039091A903F3
:102F10000C944B170F931F93CF93DF938091A903CA
:102F200082958F7009F05DC08091A603882309F413
:102F300058C080917203109173036091A403709143
:102F4000A503C091A703D091A80391E06F3F09F0BA
:102F500090E0292F06E0811709F443C0209721F063
:102F60007F3F21F030E003C031E001C0322F90E01C
:102F700030FD34C0089FF001099FF00D1124DF01DE
:102F8000AC58BC4F11963C911197371327C03C9118
:102F9000361324C012963C91129731111FC013961C
:102FA0004D915C9114974C1B5D0B483C5105B0F45E
:102FB0008091A9038F7080618093A903E758FC4F2B
:102FC00080818F708061808384EA93E00E94A613E1
:102FD000DF91CF911F910F910C945B170196877031
:102FE000BACFDF91CF911F910F9108959F92AF9229
:102FF000BF92CF92DF92EF92FF920F931F93CF93E6
:10300000DF93CDB7DEB761970FB6F894DEBF0FBE82
:10301000CDBF8C0185E0F801DE011D9601900D9277
:103020008A95E1F7F80140815181F280C380D48014
:103030009091A4036091A5032091A7033091A80368
:103040002115310531F06F3F31F481E09F3F19F4D4
:1030500003C081E001C080E0F82FF1709F2E80FD59
:1030600052C184EAA82E83E0B82EE090A603F601B0
:10307000E21BF30BEE2009F4E8C08091A903E83CC1
:10308000F10508F0A4C0282F207F09F053C0561383
:1030900013C0491311C0EF2CF1100EC08F70806166
:1030A0008093A9030E947C17C5010E94A6138091FA
:1030B000A903F80185835BC1C114D10431F05F3FDE
:1030C00031F481E04F3F19F403C081E001C080E09A
:1030D00080FD03C081E08F2502C080E090E0F82FE2
:1030E000F170EF2E80FF1CC080917203209173035A
:1030F00036E0821709F418C190E0389FF001399F3B
:10310000F00D1124EC58FC4F6181561306C060810C
:10311000461303C06281F61203C001968770E9CF9F
:10312000EF2CFF2009F423C18091A90381608093D3
:10313000A90362C0561306C0491304C0F11002C0AF
:10314000F801A7C04D875E87FF867C2DD98AC88A83
:103150006F2D89890E94DE16882399F1FF2089F15D
:103160002091A903822F82958F7090E0029774F0CE
:103170008091A4039091A50398878F831986DB869D
:10318000CA862C87CE0107960E94A61386E0F80116
:10319000A4EAB3E001900D928A95E1F70E948A17A4
:1031A0000E947C1711C0561749F14D875E87FF8634
:1031B0007C2DD98AC88A6F2D89890E94DE168111DB
:1031C0002CC0C8010E94A613EE24E394D0C0282F7F
:1031D000207F49F77C2DD98AC88A6F2D89890E9462
:1031E0003C1784EA93E00E94A61386E0F501119251
:1031F0008A95E9F70E947C17E12CB9C04913D5CF15
:10320000F110D3CFF8018583C8010E94A61386E090
:10321000F50111928A95E9F7AAC0FF2091F2209159
:10322000A903822F82958F7090E002970CF4AECFA5
:103230008091A4039091A5039A8389831B82DD82E8
:10324000CC822E83CE0101969FCFE83CF10508F099
:103250004BC0EF2CFF2009F4B4CF561330C04913F4
:103260002EC02091A90320FD21C0822F82958F704E
:10327000482F50E041155105C9F0F80125834F3022
:10328000510541F08F5F982F9295907F822F8F701C
:10329000892B8583C8010E94A61386E0F801A4EA61
:1032A000B3E001900D928A95E1F72AC086E0F8011B
:1032B000A4EAB3E001900D928A95E1F758C04D87DA
:1032C0005E87FF867C2DD98AC88A6F2D89890E94E6
:1032D000DE1681115BCF8091A90381608093A903E1
:1032E000C8010E94A61343C07C2DD98AC88A6F2DBD
:1032F00089890E943C1786E0F50111928A95E9F7C9
:103300000E947C1734C0FF2009F45BCF4D875E8795
:10331000FF867C2DD98AC88A6F2D89890E94DE1686
:10332000882309F44ECF32CF7C2DD98AC88A6F2DDD
:1033300089890E942E1C292F22952F70223028F473
:103340009F7039F0811105C00BC0243028F49F70A4
:1033500049F4805E883020F0C8010E94A6139E2C9C
:10336000E92C05C0F8019581907F99F7F9CF8E2D52
:1033700061960FB6F894DEBF0FBECDBFDF91CF913F
:103380001F910F91FF90EF90DF90CF90BF90AF9083
:103390009F9008951F93CF93DF93CDB7DEB72C97FF
:1033A0000FB6F894DEBF0FBECDBF4F835887698735
:1033B0007A878B879C87CE0107960E94F617882311
:1033C000D1F09F8188852A853B85232B31F08F3F63
:1033D00031F481E09F3F19F403C081E001C080E037
:1033E00080FD47C04F81588569857A858B859C858E
:1033F0000E944B173EC086E0FE013796DE01119613
:1034000001900D928A95E1F7FF81E8856A857B85B9
:103410006115710531F0EF3F31F481E0FF3F19F4A0
:1034200003C081E001C080E080FD23C020917303D0
:1034300030E0C9010196877099274091720350E0EE
:1034400084179507F1F1F983EA837D836C8396E015
:10345000929FD001939FB00D1124AC58BC4FFE0138
:10346000319601900D929A95E1F7809373030E9433
:103470005B1716E08091720390917303891771F1C5
:10348000189FC00111248C589C4F0E94F617882366
:1034900029F1E09172031E9FF0011124EC58FC4FBA
:1034A0004081518162817381848195810E944B1793
:1034B0008091720390E00196877099278093720340
:1034C000D9CF0E94A2131092730310927203E4EA00
:1034D000F3E086E0DF011D928A95E9F72C960FB69E
:1034E000F894DEBF0FBECDBFDF91CF911F9108953D
:1034F000DF92EF92FF920F931F93CF93DF93FC0124
:10350000892B09F488C0E12CF12CDD24D394EF0140
:1035100021968491853709F460C058F4843708F007
:103520004EC0843008F068C08130D1F0823071F133
:1035300072C0883709F45BC050F4863709F453C071
:10354000873709F068C08E2D0E94FD1C52C09CE791
:10355000980F903708F05FC08F770E9426134EC0F7
:103560008F010E5F1F4FFE01849190E2980F9830FB
:1035700050F48770FD2D01C0FF0F8A95EAF78F2F59
:103580000E94031D15C00E948F1214C08F010E5F90
:103590001F4FFE01849190E2980F983068F4877075
:1035A000FD2D01C0FF0F8A95EAF78F2F0E94091D9C
:1035B0000E942A1DE80122C00E942613FBCFCF01E2
:1035C0000296FE01C491CC2361F0EFE9FFE0319750
:1035D000F1F700C00000C150F6CFCF010296FE0106
:1035E000F490EC010BC00E94ED1CE82E07C00E9475
:1035F000001D0E942A1D02C00E948F128F2D882359
:1036000041F0EFE9FFE03197F1F700C00000815091
:10361000F6CFFE017CCFDF91CF911F910F91FF90EC
:10362000EF90DF90089560932A0470932B048093A9
:103630002C0490932D040C94781D089560932E040F
:1036400070932F0480933004909331040C94771D71
:103650000F931F9300912E0410912F04209130049A
:1036600030913104602B712B822B932B60932E04AD
:1036700070932F0480933004909331041F910F9125
:103680000C94771D0F931F9300912E0410912F041B
:1036900020913004309131046023712382239323DD
:1036A00060932E0470932F04809330049093310420
:1036B0001F910F910C94771D0F931F9300912E046F
:1036C00010912F042091300430913104602771272C
:1036D0008227932760932E0470932F0480933004E5
:1036E000909331041F910F910C94771D60E070E06E
:1036F000CB010C94131B0F931F9341E050E060E04B
:1037000070E08A019B0104C0000F111F221F331FAC
:103710008A95D2F7C901B8011F910F910C94131B20
:103720000F931F9341E050E060E070E004C0440F4D
:10373000551F661F771F8A95D2F780912A049091B2
:103740002B04A0912C04B0912D048A019B01082B1D
:10375000192B2A2B3B2BC901B8011F910F910C94F7
:10376000131B0F931F9341E050E060E070E004C032
:10377000440F551F661F771F8A95D2F740955095C5
:103780006095709580912A0490912B04A0912C044F
:10379000B0912D048A019B01082319232A233B237E
:1037A000C901B8011F910F910C94131B0F931F9324
:1037B00041E050E060E070E004C0440F551F661F18
:1037C000771F8A95D2F780912A0490912B04A091BB
:1037D0002C04B0912D048A019B01082719272A2760
:1037E0003B27C901B8011F910F910C94131B0F9334
:1037F0001F9300912A0410912B0420912C043091E6
:103800002D04602B712B822B932B1F910F910C9405
:10381000131B0F931F9300912A0410912B042091E6
:103820002C0430912D0460237123822393231F9154
:103830000F910C94131B0F931F9300912A04109166
:103840002B0420912C0430912D04602771278227AE
:1038500093271F910F910C94131B08958F929F92A1
:10386000AF92BF92DF92EF92FF920F931F93CF938D
:10387000DF9300D000D01F92CDB7DEB76B837C837F
:103880008D838A018C819D81892B31F01F3F31F41A
:1038900081E04F3F19F403C081E001C080E080FF68
:1038A00003C080E090E04DC08B818823D1F18090EF
:1038B0002A0490902B04A0902C04B0902D048091A9
:1038C0002E0490912F04A0913004B0913104882AE5
:1038D000992AAA2ABB2A8FE1E82EF12CD501C4012E
:1038E0000E2C04C0B695A795979587950A94D2F7A4
:1038F00080FD06C081E0E81AF10880F7D12C07C0EE
:10390000DE2CB8018E2D0E946C1E019799F388E081
:10391000189FF0011124E655FC4FE00FF11DD082F5
:1039200009C088E0189FF0011124E655FC4FE00F14
:10393000F11DD08009831A8369817A818D2D0E94BF
:103940006C1E0F900F900F900F900F90DF91CF9102
:103950001F910F91FF90EF90DF90BF90AF909F90DD
:103960008F9008952091110130911201F901329642
:103970009FEF40E05191851789F09F3F19F4511155
:1039800001C0942F4F5F4630A9F79F3F39F0F901EE
:10399000E90FF11D97FDFA95828308950895E0914E
:1039A0001101F09112019F012A5F3F4F928189130B
:1039B00001C012823196E217F307C1F7089581E042
:1039C00090E0E0911101F0911201E80FF91F1082CF
:1039D000019688309105A9F7089580913C040895D7
:1039E00090913C04892B80933C040895809590919C
:1039F0003C04892380933C04089580933C040895FB
:103A000010923C04089590913B04892B80933B04D1
:103A10000895809590913B04892380933B040895F9
:103A200010923B040895809332040895109232045A
:103A300008958091110190911201FC0131969C0131
:103A4000285F3F4F80E0919191118F5FE217F3075C
:103A5000D1F70895E0911101F091120180913C0499
:103A60008083E0911101F0911201908180913B04DB
:103A7000892B808380913204882361F0E0911101C9
:103A8000F09112019081892B80830E94191D811170
:103A90001092320480911101909112010C94A410A3
:103AA000909339018093380108958295982F9373EC
:103AB00044E0949F900111248C7C86958695282B58
:103AC000822F8575880F2A7A2695822B089508956E
:103AD000CF93DF9300D000D01F92CDB7DEB70F9009
:103AE0000F900F900F900F90DF91CF910895089550
:103AF00008950C94FB1180E0089580915204843065
:103B000021F110923E0420E488E190E00FB6F89491
:103B1000A895809360000FBE2093600083B7817FDB
:103B2000846083BF83B7816083BF7894889583B7AF
:103B30008E7F83BF0FB6F894A8958091600088614E
:103B400080936000109260000FBE0895CF930E9492
:103B500047120E940C070E944812C0E08C2F0E945E
:103B6000BB07811104C0CF5FC031C1F701C081E044
:103B7000CF9108950E94FD110C94A2131F920F92F1
:103B80000FB60F9211248F939F93AF93BF938091A1
:103B90003E04811113C080913F0490914004A09194
:103BA0004104B09142044196A11DB11D80933F0490
:103BB00090934004A0934104B0934204BF91AF910D
:103BC0009F918F910F900FBE0F901F90189582E0DC
:103BD00084BD93E095BD9AEF97BD80936E000895E4
:103BE0002FB7F89480913F0490914004A091410434
:103BF000B09142042FBF08952FB7F89460913F040D
:103C00007091400480914104909142042FBF089527
:103C10009C014FB7F89480913F0490914004A0918B
:103C20004104B09142044FBF821B930B08957894D6
:103C30001F920F920FB60F9211248F939F93AF9301
:103C4000BF9380913F0490914004A0914104B091B2
:103C500042040196A11DB11D80933F04909340043E
:103C6000A0934104B0934204BF91AF919F918F9173
:103C70000F900FBE0F901F9018950E942F0FF89471
:103C800087E797E7909301088093000887E090EB1F
:103C9000DC0180935B0490935C04A0935D04B0937B
:103CA0005E049CE088E10FB6F894A89580936000CC
:103CB0000FBE90936000FFCFE82FF0E088E0989F60
:103CC000E00DF11D1124E052FE4F8491982F929542
:103CD0009F708F7097700895CF93C82FCB010E946B
:103CE0005C1E40E1949F90011124282B203831055F
:103CF0001CF080E090E016C09770E92FF0E098E0AB
:103D0000C99FE00DF11D112494E0EE0FFF1F9A955D
:103D1000E1F78F70E80FF11DEE0FFF1FE052FF4F2C
:103D200085919491CF91089580E090E00895089551
:103D30008091450480FF0BC06091160185E0689F6B
:103D4000B001112475956795759567952BC081FF16
:103D500009C06091160185E0689FB0011124759536
:103D6000679520C082FF07C06091160185E0689FBB
:103D7000B001112417C0909146049923D1F06091AD
:103D80001501961788F72091160185E0289F90016C
:103D90001124929FA001939F500D112470E0CA013D
:103DA0000E9459266038710540F46115710519F4B7
:103DB00006C065E070E0862F08958FE7089581E0E2
:103DC00008958091450480FF08C06091140170E05F
:103DD000759567957595679521C081FF06C06091BF
:103DE000140170E07595679519C082FF04C0609159
:103DF000140170E010C090914604992399F06091ED
:103E000013019617A0F780911401899FC001112416
:103E100070E00E9459266038710540F46115710503
:103E200019F406C061E070E0862F08958FE70895C9
:103E300081E00895803F21F40E94981E819504C07E
:103E4000813F29F40E94981E809349040895823F7F
:103E500021F40E94981E819504C0833F29F40E949A
:103E6000981E809348040895893F19F40E94E11E2A
:103E700005C08A3F31F40E94E11E819580934A0477
:103E800008958B3F21F40E94E11E819504C08C3F70
:103E900029F40E94E11E80934B040895843F21F48D
:103EA00080914704816017C0853F21F480914704C9
:103EB000826011C0863F21F48091470484600BC06A
:103EC000873F21F480914704886005C0883F31F422
:103ED0008091470480618093470408958D3F21F4C9
:103EE0008091450481600BC08E3F21F48091450490
:103EF000826005C08F3F29F48091450484608093DF
:103F000045040895803F39F48091490487FF6CC0CF
:103F10001092490469C0813F29F480914904181620
:103F2000BCF362C090914804823F29F497FF5CC0C3
:103F30001092480459C0833F19F41916CCF354C0A9
:103F4000893F41F480914A0418160CF04DC010923C
:103F50004A044AC08A3F29F480914A0487FF44C03A
:103F6000F6CF8B3F39F480914B0487FF3DC0109210
:103F70004B043AC08C3F29F480914B041816BCF3D3
:103F800033C0843F21F4809147048E7F17C0853F62
:103F900021F4809147048D7F11C0863F21F48091E8
:103FA00047048B7F0BC0873F21F480914704877FB4
:103FB00005C0883F31F4809147048F7E8093470489
:103FC00013C08D3F21F4809145048E7F0BC08E3F3E
:103FD00021F4809145048D7F05C08F3F29F48091A5
:103FE00045048B7F809345048091480481110EC065
:103FF0008091490481110AC080914A04811106C050
:1040000080914B04811102C0109246040895809162
:104010003D0483FF7EC08AE295E00E94DC0580912A
:1040200047041F928F9385E295E09F938F930E94A0
:10403000750683E295E00E94DC0580914804282FF4
:10404000082E000C330B3F938F9380E295E09F93F3
:104050008F930E9475068EE195E00E94DC058091A9
:104060004904282F082E000C330B3F938F938BE1CC
:1040700095E09F938F930E94750689E195E00E94D9
:10408000DC0580914A04282F082E000C330B3F9347
:104090008F9386E195E09F938F930E94750684E14C
:1040A00095E00E94DC0580914B04282F082E000C1F
:1040B000330B3F938F9381E195E09F938F930E9401
:1040C00075068EE095E00E94DC05809146041F9203
:1040D0008F938BE095E09F938F930E94750689E004
:1040E00095E00E94DC05809145041F928F9386E045
:1040F00095E09F938F930E94750683E095E00E9460
:10410000DC058DB79EB74C960FB6F8949EBF0FBED8
:104110008DBF87E494E00E94ED100E94F01D909303
:1041200044048093430408951F93CF93DF938091B9
:104130004304909144040E94081EAC0190914604EF
:10414000992321F02091170130E006C02091180139
:104150008AE0289F900111244217530708F485C074
:1041600080914804C0914904D0914A0410914B04B5
:10417000811107C0C11175C0D11173C0111171C077
:1041800074C09F3F19F09F5F90934604181624F463
:104190000E94981E809348048091480487FF05C0C0
:1041A0000E94981E8195809348041C1624F40E9456
:1041B000981E809349048091490487FF05C00E949E
:1041C000981E81958093490460914804662331F1DB
:1041D000C0914904CC2311F1062E000C770B880BFB
:1041E000990B0E94602523E333E343E35FE30E94DE
:1041F000C4250E942825609348046C2FCC0F770BB0
:10420000880B990B0E94602523E333E343E35FE3CC
:104210000E94C4250E942825609349041D1624F499
:104220000E94E11E80934A0480914A0487FF05C0E2
:104230000E94E11E819580934A04111624F40E9485
:10424000E11E80934B0480914B0487FF05C00E94C0
:10425000E11E819580934B04DF91CF911F910C94C7
:1042600007209F3F09F08FCFA0CFDF91CF911F9103
:104270000895E7E4F4E085E0DF011D928A95E9F70F
:10428000109246041092450408958DE497E00E9430
:10429000DC051F9281E08F931F9285E08F938FEF53
:1042A00096E09F938F930E9475060F900F900F904A
:1042B0000F900F900F9008958330E9F128F481302A
:1042C00061F0823009F10895853009F462C008F484
:1042D00049C0863009F474C0089580911801262FD2
:1042E00030E0280F311D2F3F310524F4680F609313
:1042F000180103C08FEF80931801809118011F925D
:104300008F9388E396E072C080911701262F30E0EA
:10431000280F311D2F3F310524F4680F60931701DA
:1043200003C08FEF80931701809117011F928F9325
:1043300086E296E05BC080911601262F30E0280FC0
:10434000311D2F3F310524F4680F6093160103C01F
:104350008FEF80931601809116011F928F9383E156
:1043600096E044C080911501262F30E0280F311DC2
:104370002F3F310524F4680F6093150103C08FEFC0
:1043800080931501809115011F928F938EEF95E018
:104390002DC080911401262F30E0280F311D2F3FB2
:1043A000310524F4680F6093140103C08FEF8093EC
:1043B0001401809114011F928F9385EE95E016C031
:1043C00080911301262F30E0280F311D2F3F31053A
:1043D00024F4680F6093130103C08FEF80931301DF
:1043E000809113011F928F938AEC95E09F938F9396
:1043F0000E9475060F900F900F900F9008958330D4
:1044000081F128F4813059F08230D1F0089585305F
:1044100009F449C0B8F1863009F456C00895809176
:104420001801681720F4861B8093180102C01092AF
:104430001801809118011F928F938BEB95E054C067
:1044400080911701681720F4861B8093170102C022
:1044500010921701809117011F928F9389EA95E0BE
:1044600043C080911601681720F4861B80931601C3
:1044700002C010921601809116011F928F9386E957
:1044800095E032C080911501681720F4861B809357
:10449000150102C010921501809115011F928F9392
:1044A00081E895E021C080911401681720F4861BF3
:1044B0008093140102C010921401809114011F9284
:1044C0008F9388E695E010C080911301681720F45F
:1044D000861B8093130102C0109213018091130177
:1044E0001F928F938DE495E09F938F930E947506A2
:1044F0000F900F900F900F900895CF93C82F1F9299
:104500008F9382E598E09F938F930E94750681E0D8
:1045100090E0A0E0B0E0BC01CD0104C0660F771FC1
:10452000881F991FCA95D2F70E941E1B0F900F90EB
:104530000F900F90CF910C94A213CF93873288F5F0
:104540008E3108F00BC18E3009F487C0D8F4873063
:1045500009F460C08B3009F44FC0863009F002C105
:1045600080913D04817F8E7F80933D0487E598E0B4
:104570000E94DC0588E09BE00E94DC0581E08093DE
:104580004D0446C0863109F4B0C020F4803109F4EE
:104590007AC0E8C0893109F491C08B3109F449C06F
:1045A000E1C0883349F150F4893209F4D5C085332C
:1045B00009F4D2C0873209F0D5C0CEC0833409F4E3
:1045C000CBC028F48A3308F4CDC08953C8C08834DE
:1045D00009F0C8C00E94A21387EF9AE00E94DC0590
:1045E0002FEF83ED90E3215080409040E1F700C031
:1045F00000000E943D1E0CC08EE798E041C08EED89
:104600009AE00E94DC0580913D04816080933D0426
:10461000C1E0ADC080913D04C82FC17080FFEFCFD5
:104620008AEE9AE00E94DC0580913D04817F8E7FB6
:104630003FC090913D0491FBCC27C0F981E0C82791
:10464000892FC0FB81F980933D04CC2319F081EDC3
:104650009AE029C083EC9AE013C090913D0492FB4C
:10466000CC27C0F981E0C827892FC0FB82F980934D
:104670003D04CC2319F084EB9AE015C084EA9AE05B
:104680000E94DC05C5CF90913D0493FBCC27C0F977
:1046900081E0C827892FC0FB83F980933D04CC2398
:1046A00051F088E99AE00E94DC0580913D04816028
:1046B00080933D045CC08BE89AE0E2CF8CE79AE0FF
:1046C0000E94DC058CE49AE00E94DC0586E09AE01A
:1046D0000E94DC058DED99E00E94DC0587EA99E0F7
:1046E0000E94DC058CE799E0CBCF8EE699E00E9432
:1046F000DC050E9498101F928F9384E599E09F93A8
:104700008F930E947506809110011F928F938DE305
:1047100099E09F938F930E94750680915A031F9290
:104720008F938AE299E09F938F930E9475060E946F
:10473000FC1D9F938F937F936F9383E199E09F93E9
:104740008F930E9475068DB79EB742960FB6F89468
:104750009EBF0FBE8DBF5CCF80E001C08D510E9417
:104760007D2256CF81E199E00E94DC05C0E08C2FCC
:10477000CF91089580E008950C94BA230F931F936E
:10478000CF93C82F80914D048130B1F020F082305A
:1047900009F45BC052C160E070E08CE090E00E94E0
:1047A000FF11892BC9F4E0911101F0911201808170
:1047B000843409F044C110C060E070E08CE090E007
:1047C0000E94FF118C01892B39F4E0911101F091C5
:1047D00012018081843461F48C2F0E94BC238111EA
:1047E00004C08C2F0E949D222EC081E090E02BC03F
:1047F0008C2F0E94BA23811124C1C431E1F070F4DE
:10480000CB3081F0C031D1F40E9445218AE498E098
:104810000E94DC0582E080934D0413C1C93259F037
:10482000C83361F487E598E00E94DC058EE498E0E7
:104830000E94DC0506C110924D0404C088E498E093
:104840000E94DC05802F8170FFC0C43228F5CE3174
:1048500008F0C1C0CB30A1F1D0F4C73009F0D3C00B
:104860008EE18093180182E3809317018AE08093A0
:10487000160184E18093150188E08093140188E299
:10488000809313018EEE96E00E94DC05BFC0C33119
:1048900049F1C431C1F0B7C0CB3409F4A9C028F440
:1048A000C93289F0C83361F0AEC0C13509F49EC089
:1048B000C23509F499C0CE3409F0A5C06AE09EC0A3
:1048C0000E944521A3C080914C04882319F01092C6
:1048D0004C049CC08BEF96E00E94DC0581E0809345
:1048E0004D04B2C085ED96E00E94DC0583EC96E0B5
:1048F0000E94DC05809118011F928F9380EC96E056
:104900009F938F930E9475068EEB96E00E94DC05C4
:104910008CEA96E00E94DC05809117011F928F932C
:1049200089EA96E09F938F930E94750687EA96E046
:104930000E94DC0588E996E00E94DC058091160162
:104940001F928F9385E996E09F938F930E9475063F
:1049500083E996E00E94DC0582E896E00E94DC058F
:10496000809115011F928F938FE796E09F938F930D
:104970000E9475068DE796E00E94DC0588E696E0C9
:104980000E94DC05809114011F928F9385E696E0CA
:104990009F938F930E94750683E696E00E94DC0544
:1049A0008CE496E00E94DC05809113011F928F93A6
:1049B00089E496E09F938F930E94750687E496E0C2
:1049C0000E94DC058DB79EB748960FB6F8949EBF3F
:1049D0000FBE8DBF1BC0CE51EC2FF0E0E25DFE4F4D
:1049E000808180934C0412C061E003C061E006C086
:1049F0006AE080914C040E945C2108C080914C04C4
:104A00000E94FF2103C08CEE96E013C080914C04FD
:104A1000882369F01F928F9386EE96E09F938F9381
:104A20000E9475060F900F900F900F9004C083EEB8
:104A300096E00E94DC0581E007C010924D0480E002
:104A400003C001E010E0FECECF911F910F910895B9
:104A50000E942F256894B1110C94BE2508950E94E0
:104A6000A32588F09F5798F0B92F9927B751B0F038
:104A7000E1F0660F771F881F991F1AF0BA95C9F7E2
:104A800014C0B13091F00E94BD25B1E008950C949E
:104A9000BD25672F782F8827B85F39F0B93FCCF351
:104AA000869577956795B395D9F73EF4909580955F
:104AB000709561957F4F8F4F9F4F0895E89409C07F
:104AC00097FB3EF490958095709561957F4F8F4F41
:104AD0009F4F9923A9F0F92F96E9BB279395F69557
:104AE000879577956795B795F111F8CFFAF4BB0FD5
:104AF00011F460FF1BC06F5F7F4F8F4F9F4F16C039
:104B0000882311F096E911C0772321F09EE8872FC2
:104B1000762F05C0662371F096E8862F70E060E07E
:104B20002AF09A95660F771F881FDAF7880F9695F7
:104B3000879597F9089557FD9058440F551F59F0E0
:104B40005F3F71F04795880F97FB991F61F09F3F7A
:104B500079F087950895121613061406551FF2CFA3
:104B60004695F1DF08C0161617061806991FF1CFF3
:104B700086957105610508940895E894BB2766271A
:104B80007727CB0197F908950E94D7250C944826E2
:104B90000E943A2638F00E94412620F0952311F019
:104BA0000C9431260C94372611240C94BE250E94B7
:104BB0009B2570F3959FC1F3950F50E0551F629FA1
:104BC000F001729FBB27F00DB11D639FAA27F00D66
:104BD000B11DAA1F649F6627B00DA11D661F829F8D
:104BE0002227B00DA11D621F739FB00DA11D621F72
:104BF000839FA00D611D221F749F3327A00D611D8F
:104C0000231F849F600D211D822F762F6A2F112470
:104C10009F5750409AF0F1F088234AF0EE0FFF1FA3
:104C2000BB1F661F771F881F91505040A9F79E3FFA
:104C3000510580F00C9431260C94BE255F3FE4F3BF
:104C4000983ED4F3869577956795B795F795E79550
:104C50009F5FC1F7FE2B880F911D9695879597F959
:104C6000089597F99F6780E870E060E008959FEFEE
:104C700080EC089500240A941616170618060906F3
:104C8000089500240A9412161306140605060895C2
:104C9000092E0394000C11F4882352F0BB0F40F44A
:104CA000BF2B11F460FF04C06F5F7F4F8F4F9F4F8A
:104CB000089597FB072E16F4009407D077FD09D0CE
:104CC0000E94732607FC05D03EF4909581959F4F76
:104CD0000895709561957F4F0895EE0FFF1F059021
:104CE000F491E02D0994AA1BBB1B51E107C0AA1F38
:104CF000BB1FA617B70710F0A61BB70B881F991F7D
:104D00005A95A9F780959095BC01CD010895F89426
:024D1000FFCFD3
:104D12000551020000FF4D08DD08BA08840850085A
:104D22000133042808140A321E404D36226F042231
:104D320004EC03CA0356036F038803A103000102B4
:084D420003040506070809003F
:00000001FF
